:1000000040280339A4000310A40DA40D83161F0873
:100010008F3930389F0083121F08F33924040138C8
:100020009F00323027209F149F181428A7011E0814
:10003000A6003C28A301A200FF30A207031CA307CF
:10004000031C3C280330A100DF3028201C28A1011C
:10005000E83EA000A109FC30031C3128A0070318CA
:100060002E28A0070000A10F2E2820183728A01C3A
:100070003B2800003B280800831383120313080069
:1000800083161F109F141F119F110515851205124D
:10009000851505108312851205120510AA01051495
:1000A0000130A300F4301B2001300120AA000230EF
:1000B0002A02031C5C2861280130A300F4301B20B5
:1000C00054280130A300F4301B200516851D692833
:1000D00081280514A801A90102302902031C7628F1
:1000E000031D7E28D130280203187E28EA30A300A1
:1000F00060301B20A80A0319A90F6C2805120510EF
:1001000098280514A801A90101302902031C8E2892
:10011000031D96286930280203189628EA30A300A8
:1001200060301B20A80A0319A90F842805120510A6
:1001300085160330A300E8301B2085120730A3008A
:08014000D0301B209828A328F1
:02400E00843FED
:00000001FF
